:020000040000FA
:080000000000000000000000F8
:080008001E2133213F2D211EB2
:080010001E3F2D3F21333F1E6E
:08001800000A1B1F1F0E04006B
:0800200000040E1F1F0E040076
:08002800000E04151F15040E63
:0800300000040E1F1F1F040E47
:0800380000000C1E1E0C00006C
:080040003F3F332121333F3F14
:0800480000000C12120C000074
:080050003F3F332D2D333F3FEC
:080058000703050C12120C0055
:08006000000E11110E040E0444
:080068000F090F0808183818F1
:080070001F111F1111133330A1
:0800780004150E1B1B0E1504FC
:080080000010181C1E1C1810D2
:080088000002060E1E0E060226
:08009000040E1F04041F0E04FE
:08009800000A0A0A0A000A002E
:0800A000000F1515150D0505F3
:0800A800000E100C120C021CEA
:0800B00000000000001E1E000C
:0800B800040E1F041F0E041FBB
:0800C00000040E1F04040404F7
:0800C80000040404041F0E04EF
:0800D000000004061F060400F5
:0800D8000000040C1F0C0400E1
:0800E0000000001010101F00C9
:0800E800000012213F2112006B
:0800F0000000040E1F1F0000B8
:0800F80000001F1F0E040000B0
:080100000000000000000000F7
:080108000004040404000400DB
:08011000000A0A0000000000D3
:08011800000A1F0A0A1F0A0079
:0801200000040F140E051E047B
:080128000000191A040B13007A
:0801300000040A040B120D008B
:080138000004080000000000B3
:080140000002040404040200A3
:0801480000040202020204009F
:0801500000000A041F040A006C
:08015800000004041F04040070
:08016000000000000004040887
:08016800000000001F00000070
:08017000000000000000040083
:08017800000001020408100060
:08018000000E131515190E0005
:0801880000040C0404040E0045
:08019000000E11010E101F000A
:08019800001F020601110E0018
:0801A0000002060A121F020012
:0801A800001F101E01110E00E2
:0801B000000E101E11110E00DB
:0801B800001F01020404040011
:0801C000000E110E11110E00DA
:0801C800000E11110F010E00E1
:0801D00000000004000004001F
:0801D80000000400000404080B
:0801E000000002040804020003
:0801E8000000001F001F0000D1
:0801F0000000080402040800ED
:0801F800000E110204000400D6
:08020000000E111717100E008B
:08020800000E11111F1111007D
:08021000001E111E11111E0059
:08021800000E111010110E0080
:08022000001E090909091E0076
:08022800001F101E10101F0042
:08023000001F101E1010100049
:08023800000E111017110E0059
:080240000011111F1111110042
:08024800000E040404040E0082
:080250000001010101110E0083
:08025800001214181412110029
:080260000010101010101F0027
:0802680000111B15111111001A
:0802700000111915151311000E
:08027800000E111111110E001E
:08028000001E11111E101000F8
:08028800000E111115120D000A
:08029000001E11111E121100E5
:08029800000E100E01110E0012
:0802A000001F04040404040023
:0802A8000011111111110E00EB
:0802B00000111111110A0400F4
:0802B8000011111515150A00D3
:0802C00000110A04040A1100F8
:0802C8000011110A04040400F6
:0802D000001E020408101E00CC
:0802D800000E080808080E00E2
:0802E0000000100804020100F7
:0802E800000E020202020E00EA
:0802F00000040A1100000000E7
:0802F800000000000000003FBF
:080300000008040000000000E9
:0803080000000E010F110F00AF
:080310000010101E11111E0067
:0803180000000E1010100E0091
:080320000001010F11110F0093
:0803280000000E111E100F0071
:080330000006080C0808080093
:0803380000000F11110F010E6E
:080340000010101E1111110044
:080348000004000C04040E0087
:08035000000200020202120C7F
:08035800001012141814120029
:08036000000C040404040E006B
:0803680000001A15151515001F
:0803700000001E111111110023
:0803780000000E1111110E002E
:0803800000001E11111E1010F7
:0803880000000F11110F01012B
:0803900000000E101010100017
:0803980000000E100E011E0012
:0803A00000081C080808060013
:0803A8000000111111110E00FB
:0803B000000011110A0A04000B
:0803B8000000111115150A00E7
:0803C0000000110A040A1100FB
:0803C80000001111110F010EDC
:0803D00000001F0204081F00D9
:0803D8000002040418040402F1
:0803E0000004040400040404FD
:0803E8000008040403040408EA
:0803F000000A140000000000E7
:0803F8000000040A111F0000BF
:08040000000709111F11110092
:08040800001F101E11111E005F
:08041000001E111E11111E0057
:08041800001F1010101010006D
:08042000000E121212123F211E
:08042800001F101E10101F0040
:080430000015150E0E15150054
:08043800000E110601110E0077
:0804400000111315151911003C
:08044800041511131519110030
:080450000011121C1211110031
:08045800000709090909110060
:0804600000111B151111110020
:080468000011111F1111110018
:08047000000E111111110E0024
:08047800001F11111111110008
:08048000001E11111E101000F6
:08048800000E111010110E000E
:08049000001F04040404040031
:08049800001111110F010E000B
:0804A000000E1515150E0400F5
:0804A80000110A04040A11000E
:0804B0000012121212121F01CA
:0804B800001111110F010100F8
:0804C0000015151515151F00AC
:0804C8000015151515151F01A3
:0804D0000018080E09090E00D6
:0804D8000011111D13131D009A
:0804E0000010101E11111E0096
:0804E800001E010F01011E00BE
:0804F0000012151D1515120084
:0804F800000F11110F091100A2
:0805000000000E010F110F00B5
:0805080000001F101E111E006F
:0805100000001E111E111E0067
:0805180000001F10101010007C
:0805200000000E1212123F212F
:0805280000000E111E100E0070
:08053000000015150E15150061
:0805380000000E1106110E0077
:08054000000011131519110050
:08054800040411131519110040
:08055000000011121C12110041
:08055800000007090909110068
:080560000000111B1511110030
:08056800000011111F11110028
:0805700000000E1111110E0034
:0805780000001F111111110018
:080580002A0015002A001500F5
:080588002A152A152A152A156F
:080590002A3F153F2A3F153FE9
:0805980004040404040404043B
:0805A000040404043C040404FB
:0805A8000404043C043C0404BB
:0805B0000A0A0A0A3A0A0A0AC3
:0805B800000000003E0A0A0ADF
:0805C0000000003C043C0404AF
:0805C8000A0A0A3A023A0A0A83
:0805D0000A0A0A0A0A0A0A0AD3
:0805D8000000003E023A0A0A8D
:0805E0000A0A0A3A023E00007B
:0805E8000A0A0A0A3E000000A5
:0805F0000404043C043C00007B
:0805F800000000003C040404B3
:080600000404040407000000DB
:08060800040404043F0000009B
:08061000000000003F04040497
:080618000404040407040404B7
:08062000000000003F00000093
:08062800040404043F0404046F
:0806300004040407040704049C
:080638000A0A0A0A0B0A0A0A69
:080640000A0A0A0B080F000072
:080648000000000F080B0A0A74
:080650000A0A0A3B003F00000A
:080658000000003F003B0A0A0C
:080660000A0A0A0B080B0A0A42
:080668000000003F003F00000C
:080670000A0A0A3B003B0A0ADA
:080678000404043F003F0000F0
:080680000A0A0A0A3F0000000B
:080688000000003F003F0404E4
:08069000000000003F0A0A0A05
:080698000A0A0A0A0F00000023
:0806A000040404070407000034
:0806A800000000070407040430
:0806B000000000000F0A0A0A15
:0806B8000A0A0A0A3B0A0A0AB9
:0806C0000404043F043F04049C
:0806C800040404043C000000DE
:0806D00000000000070404040F
:0806D8003F3F3F3F3F3F3F3F22
:0806E000000000003F3F3F3F16
:0806E80038383838383838384A
:0806F0000707070707070707CA
:0806F8003F3F3F3F00000000FE
:0807000000001E111E10100084
:0807080000000E1110110E009B
:0807100000001F0404040400B2
:08071800000011110F010E0099
:0807200000000E15150E040087
:080728000000110A040A11008F
:080730000000121212121F0159
:08073800000011110F01010086
:080740000000151515151F003E
:080748000000151515151F0135
:08075000000018080E090E005C
:08075800000011111D131D002A
:08076000000010101E111E0024
:0807680000001E010F011E003C
:08077000000012151D15120016
:0807780000000F110F09110030
:080780000A1F101F10101F00DA
:080788000A000E111E100E0004
:08079000000F101E10100F00F5
:0807980000000F101E100F00FD
:0807A0000A0E040404040E001B
:0807A8000A000C0404040E0019
:0807B000041511110F010E00E8
:0807B800040411110F010E00F1
:0807C000000C12120C000000F5
:0807C8000000000A040A000011
:0807D00000000000040000001D
:0807D80000010102120C0400F3
:0807E0000013131A1612120097
:0807E8000C1204081E000000C1
:0807F0000000000E0E0E0000D7
:0807F8000000000000000000F9
:00000001FF
